:100000000C9420020C943D020C943D020C943D0291
:100010000C943D020C943D020C943D020C943D0264
:100020000C943D020C943D020C94421E0C94141F3F
:100030000C9413190C943D020C943D020C943D0257
:100040000C943D020C943D020C943D020C943D0234
:100050000C943D020C949B190C943D020C943D02AF
:100060000C943D020C943D020C943D020C943D0214
:100070000C943D020C943D020C943D020C943D0204
:100080000C943D020C943D020C943D020C943D02F4
:100090000C943D020C943D020C943D020C943D02E4
:1000A0000C943D020C943D020C943D02FF04FF04AD
:1000B0002B052B059305B105C906C906BC055506D8
:1000C00066066606811FA81FA020A81FA020F41F97
:1000D0001720A0206E207D2029003B003D003F001E
:1000E0004100430045004700000056003A003C0034
:1000F0003E00400042004400460048000000570017
:1001000035001F0021002300250027002E00490094
:100110004B0054001E0020002200240026002D0069
:100120002A004A00530055002B001A0015001C003D
:100130000C00130030004C004E006000140008005A
:100140001700180012002F0031004D005F00610001
:100150003900160009000B000E00330028000000D3
:100160005C005E00040007000A000D000F00340070
:10017000000000005D006700E1001B001900110095
:10018000360038000151520059005B001D00060086
:10019000050010003700E100000000005A00580080
:1001A000E000E200000000000000E60076005000E1
:1001B0004F006300E30031002C0000000000E70066
:1001C000E400510062000000010001000100010094
:1001D0000100010001000100000001000100010018
:1001E0000100010001000100010001000000010008
:1001F000005C01000100010001000100010001009C
:1002000001000100010001000100010001000100E6
:1002100001000100010001000100010001000100D6
:1002200001000100010001000100010001000100C6
:1002300001000100010001000100010001000100B6
:1002400001000100010001000100010001000000A7
:100250000100010001000100010001000100010096
:100260000000000001000100010001000100010088
:100270000100010001000100010001000100010076
:100280000100010001000100000000000100010068
:100290000100010000000000000001000100010059
:1002A0000100010001000100010000000000010048
:1002B00001000100010000001A0341005400310058
:1002C000300031005F004200480020005000430031
:1002D00042000000220362006C0069006E006400AE
:1002E00061007300730061007300730069006E00A9
:1002F00031003100310000000403090409023B0011
:10030000020100A0FA090400000103010100092113
:1003100011010001224000070581030800010904C2
:100320000100010300000009211101000122B600B3
:10033000070582032000011201000200000008ED01
:10034000FE606001000102000105010902A10185B2
:10035000020901A1000509190129081500250195C7
:1003600008750181020501093009311581257F9544
:10037000027508810609381581257F950175088168
:1003800006050C0A38021581257F9501750881063E
:10039000C0C005010980A101850319012AB7001514
:1003A0000126B700950175108100C0050C0901A157
:1003B00001850419012AA002150126A002950175E4
:1003C000108100C005010906A1018506050719E095
:1003D00029E7150025019508750181020507190017
:1003E00029EF1500250195F0750181020508190115
:1003F0002905950575019102950175039101C005C7
:10040000010906A101050719E029E7150025019555
:1004100008750181029501750881010507190029F8
:10042000FF150026FF0095067508810005081901D3
:100430002905950575019102950175039101C0008B
:1004400011241FBECFEFDAE0DEBFCDBF11E0A0E088
:10045000B1E0E6EAF2E402C005900D92A239B107DC
:10046000D9F723E0A2E9B1E001C01D92AA30B2079A
:10047000E1F70E94DC120C9451210C940000249AA4
:10048000569A579A80FF02C05F9A01C05F9881FF19
:1004900002C02C9A01C02C9882FF02C05E9A089577
:1004A0005E98089581E0089581E008950C945402C7
:1004B00008950C9458021F93CF93DF9300D000D07F
:1004C0001F92CDB7DEB749835A836B833091950174
:1004D00089819A81311114C0662359F0222349F091
:1004E0000E940609182F682F89819A810E94AF08FF
:1004F00003C00E94DA08182F69817A81812F04C015
:100500000E94060969817A810F900F900F900F90D9
:100510000F90DF91CF911F910C944710FC01262F73
:10052000408151816281738184810C945B0281E0FE
:100530000895CF93DF93EC0160E00E948E02BE012C
:10054000DF91CF910C9459020C948D110C94891168
:1005500008950E9459070E94A8022FEF84E39CE0AF
:10056000215080409040E1F700C000000C94C11978
:100570000F931F93CF93DF938C0161E00E948E0253
:10058000EC01B8010E9456028823F1F1B801CE01B6
:100590000E945E178823C1F1B801CE010E94721536
:1005A000882391F1B801CE010E94BA16882361F127
:1005B000F8018281882309F1CB358DE5D807C1F098
:1005C00050F4C115FCE5DF0781F0CF3DDC45A9F40F
:1005D0000E943D0E19C0CC35EDE5DE0761F0CD354A
:1005E000DD4559F40E94800D08C00E94A9020CC08C
:1005F0000E94890D02C00E948C0DC801DF91CF912D
:100600001F910F910C94520280E0DF91CF911F91C6
:100610000F9108950E94F5180C9422030E9425035F
:100620000C94FB180C943F0281E008950C94140381
:100630000895CF93C82F0E9412038C2F0E94160397
:10064000CF91089580E00C9419030E94BA170C947E
:1006500019030E94BA1790919401891721F0809391
:1006600094010C9419030895CF93DF93CDB7DEB7AF
:100670002B970FB6F894DEBF0FBECDBF4F835887C0
:1006800069877A878B8761110E94CC0C9E012F5F4E
:100690003F4F86E0F90111928A95E9F785E0FE0166
:1006A0003796D90101900D928A95E1F789819A8157
:1006B0004C815D81452B31F09F3F31F491E08F3FBC
:1006C00019F403C091E001C090E090FF09C0498196
:1006D0005A816B817C818D819E810E94ED0B05C0CA
:1006E000C9010E9497028111F2CF2B960FB6F894A0
:1006F000DEBF0FBECDBFDF91CF910895FC01808199
:1007000091810E9448090895CF93882309F4A4C0D9
:10071000C82F8238C1F40E94BA1781FD9DC069E3D9
:1007200080910201909103010E94B0180E94EE0C8A
:100730002FEF81EE94E0215080409040E1F700C01F
:10074000000069E319C0833801F50E94BA1780FDE3
:1007500083C063E580910201909103010E94B0186B
:100760000E94EE0C2FEF81EE94E0215080409040EB
:10077000E1F700C0000063E5809102019091030160
:100780000E94BB18CF910C94EE0C8438C1F40E94E7
:10079000BA1782FD61C067E4809102019091030164
:1007A0000E94B0180E94EE0C2FEF81EE94E02150D1
:1007B00080409040E1F700C0000067E4DDCF8CEF9F
:1007C0008C0F813AD0F46C2F80910201909103013B
:1007D0000E943018882349F06C2F8091020190917B
:1007E00003010E94BB180E94EE0C6C2F8091020145
:1007F000909103010E94B018C5CF80E28C0F883021
:1008000048F4C77081E001C0880FCA95EAF70E94DA
:10081000AF0CB8CFEBE5EC0FE33040F4F0E0E95B70
:10082000FE4F808190E0CF910C94EE17E8E5EC0F3D
:10083000E73150F4F0E0EE0FFF1FE75EFE4F8081DE
:100840009181CF910C940418CD3E30F08C2F0E94F2
:100850006113CF910C943314CF910895882309F438
:1008600064C0823879F40E94BA1781FF5EC069E3E0
:1008700080910201909103010E94B0180E94EE0C39
:1008800069E310C08338B1F40E94BA1780FF4DC0ED
:1008900063E580910201909103010E94B0180E94CB
:1008A000EE0C63E580910201909103010E94BB1858
:1008B0000C94EE0C843879F40E94BA1782FF35C08C
:1008C00067E480910201909103010E94B0180E9498
:1008D000EE0C67E4E7CF9CEF980F913A10F4682F85
:1008E000E1CF90E2980F983050F4877091E001C00A
:1008F000990F8A95EAF7892F0E94B50CD9CF9BE50D
:10090000980F933020F480E090E00C94EE1798E577
:10091000980F973120F480E090E00C9404188D3EFD
:1009200020F00E94BC130C94331408951F93CF93AE
:10093000DF93182FEB010E948403209741F08FE989
:100940009FE00197F1F700C000002197F6CF812FBB
:10095000DF91CF911F910C942E04893319F060E040
:1009600070E002C060E570E00C949604882321F0EA
:100970000E94AF0C0C94EE0C0895882321F00E9485
:10098000B50C0C94EE0C0895CF92DF92EF92FF928B
:100990000F931F93CF93DF937C01D62FC72FFC01BA
:1009A0001281058102950F700E94A50C8823B9F071
:1009B0001123A9F08C2F807F803421F080E28D0FED
:1009C000883068F08091C80282FD09C082E00E94F0
:1009D0004E0D0E94A50C91E0D82ED92601C0D12C35
:1009E000CC2EC2948FE0C8228C2D90E08C309105E3
:1009F00008F0CFC1FC01EA5AFF4F0C94E8208C2F7D
:100A0000807FCF70882311F0C295C07F112399F0A9
:100A1000CC2309F4AAC180E28D0F883010F0D111E7
:100A200004C08C2F0E94AF0C03C08C2F0E94BF0CFF
:100A30000E94EE0C9AC18D2F0E942E04CC2309F443
:100A4000A8C180E28D0F883038F1DD2329F18C2F89
:100A50000E94C50C24C08C2F807FCF70803211F093
:100A6000C295C07FDD2319F0D130A1F13DC0809146
:100A7000C80282FF17C0112349F0CC2329F08C2F24
:100A80000E94AF0C0E94EE0C80E070C180E00E94DA
:100A90002E04CC2309F47DC18C2F0E94B50C0E943A
:100AA000EE0C77C1112371F0002341F0013031F4D5
:100AB0000E94CF0C8C2B0E94D70C6BC10E94CF0CD4
:100AC0008C2B1DC0002319F0013009F462C10E9473
:100AD000E40C25C0112321F0063008F05AC10EC0E5
:100AE000053008F056C11BC0112361F0002331F01E
:100AF000F701858180FF39C18F7085838C2F0E941B
:100B0000B60447C1002359F0D93309F03FC1FFEFC4
:100B100007EE13E0F15000401040E1F735C18C2F93
:100B20000E94BD0436C18C2F86958695837019F07E
:100B3000813061F02EC1112321F08D2F9C2F9370F5
:100B400002C080E090E00E94EE172BC1112321F03B
:100B50008D2F9C2F937002C080E090E00E940418BB
:100B600020C18D2F112319F00E94611302C00E9431
:100B7000BC130E94331415C18C2F837009F047C039
:100B800011110BC12D2F229526952770220F220FB0
:100B90006D2F6F70862F90E0A0E0B0E0022E04C0B1
:100BA000880F991FAA1FBB1F0A94D2F7D4FF10C049
:100BB0004FE050E060E070E004C0440F551F661F36
:100BC000771F2A95D2F7409550956095709503C090
:100BD00040E050E0BA01C695C695C3708A019B01FA
:100BE000082B192B2A2B3B2BC901B801C23049F025
:100BF00058F4C13019F00E94C507CFC00E94B30756
:100C0000CCC00E94D707C9C00E94B107C6C011233B
:100C100019F08C2F817001C08695882309F4BDC01E
:100C20002D2F229526952770220F220F6D2F6F7082
:100C3000862F90E0A0E0B0E0022E04C0880F991F3C
:100C4000AA1FBB1F0A94D2F7D4FF10C04FE050E098
:100C500060E070E004C0440F551F661F771F2A959F
:100C6000D2F7409550956095709503C040E050E0F4
:100C7000BA01C695C695C3708A019B01082B192B32
:100C80002A2B3B2BC901B801C23049F058F4C130BE
:100C900019F00E948A0881C00E9478087EC00E94D4
:100CA0009C087BC00E94EB0778C0CF70112339F0FD
:100CB0008C2F0E9411088D2F0E94B6046EC08D2FBC
:100CC0000E94BD048C2F0E94320867C0D23F21F1E0
:100CD00028F4D03F41F0D13FC1F043C0D33F19F1D8
:100CE000D43F79F03EC0112341F0053008F051C0E7
:100CF0008C2F8F710E9457084CC0063008F049C0F5
:100D0000F7CF8091C80282FF18C0112339F08C2FD1
:100D10008F710E9411083DC01123C9F38C2F8F7170
:100D20000E94320836C0112329F08C2F8F710E9447
:100D3000FC072FC00E94F7072CC0112349F0CF7188
:100D40008C2F0E94110863E08C2F0E94330D21C06C
:100D500081E00E944E0D0230E0F082E00E944E0DD4
:100D600018C0112331F0002391F28D2F0E948403CB
:100D700010C0002399F2D93349F41FEF27EE33E076
:100D8000115020403040E1F700C000008D2F0E943C
:100D90002E0488EF8C0D843020F40E94BA170E9434
:100DA0001903DD20C9F00E94A10C80FD15C0F701D8
:100DB00012820E949B0C0E941108C7010E940D071D
:100DC0000E949B0CDF91CF911F910F91FF90EF90AC
:100DD000DF90CF900C943208DF91CF911F910F914B
:100DE000FF90EF90DF90CF9008950F931F93CF93D4
:100DF000DF93EC01688179818A810E9453098C011B
:100E00000E94AE080E949F07B801CE010E94C40450
:100E1000DF91CF911F910F910895CF93DF93EC0154
:100E2000988189812B813C81232B31F08F3F31F4D4
:100E300081E09F3F19F403C081E001C080E080FDA4
:100E40001DC0CE010E94B802811110C00E94A50CE5
:100E50008823A1F08A81882389F08091C80282FDCD
:100E60000DC082E0DF91CF910C944E0DCE010E9417
:100E7000F506CE01DF91CF910C949902DF91CF91CD
:100E8000089580E090E00E94EE1780E090E00E94DC
:100E900004180E94CC0C0E94EE0C0E9464150C9465
:100EA000331480910201909103010E94C6180C94A2
:100EB00041070E94BC0C0C94510792959F7096308C
:100EC00079F010F4925001C09A50923068F4803F4B
:100ED00069F018F4883E40F409C0843F29F406C044
:100EE000883E20F0813F11F080E0089581E0089570
:100EF000FC01808191810E9448090E945D0708954C
:100F0000CF93DF9300D000D01F92CDB7DEB70F9004
:100F10000F900F900F900F90DF91CF910895CF9386
:100F2000DF9300D000D000D0CDB7DEB726960FB645
:100F3000F894DEBF0FBECDBFDF91CF910895089525
:100F400008950C94A0070C94A1070E94A307609336
:100F5000E5017093E6018093E7019093E8010C941A
:100F600041070C94A5070F931F930091E501109181
:100F7000E6012091E7013091E801602B712B822B73
:100F8000932B1F910F910C94A5070F931F93009122
:100F9000E5011091E6012091E7013091E80160231D
:100FA0007123822393231F910F910C94A5070F9314
:100FB0001F930091E5011091E6012091E701309126
:100FC000E80160277127822793271F910F910C94C6
:100FD000A5070C94A0070E94E9076093E1017093B4
:100FE000E2018093E3019093E4010C94410760E0F7
:100FF00070E0CB010C94EB070F931F9341E050E09E
:1010000060E070E08A019B0104C0000F111F221FE5
:10101000331F8A95D2F7C901B8011F910F910C9423
:10102000EB070F931F9341E050E060E070E004C0D5
:10103000440F551F661F771F8A95D2F78091E101F3
:101040009091E201A091E301B091E4018A019B013A
:10105000082B192B2A2B3B2BC901B8011F910F918B
:101060000C94EB070F931F9341E050E060E070E0B9
:1010700004C0440F551F661F771F8A95D2F740950D
:101080005095609570958091E1019091E201A09159
:10109000E301B091E4018A019B01082319232A236B
:1010A0003B23C901B8011F910F910C94EB070F93DB
:1010B0001F9341E050E060E070E004C0440F551F12
:1010C000661F771F8A95D2F78091E1019091E20126
:1010D000A091E301B091E4018A019B01082719273F
:1010E0002A273B27C901B8011F910F910C94EB07E8
:1010F0000F931F930091E1011091E2012091E30110
:101100003091E401602B712B822B932B1F910F9157
:101110000C94EB070F931F930091E1011091E201F2
:101120002091E3013091E401602371238223932312
:101130001F910F910C94EB070F931F930091E10106
:101140001091E2012091E3013091E40160277127C1
:10115000822793271F910F910C94EB0708952AE0A3
:10116000929F800D1124E82FE695E695E69587700D
:1011700051E001C0550F8A95EAF785E0E89FF0013C
:101180001124EA56FE4F20E030E070E04081CB01B0
:10119000022E02C0969587950A94E2F78170819598
:1011A00084278523842781932F5F3F4F2530310586
:1011B00069F708952AE0929F800D1124682F6695A3
:1011C00066956695982F977085E0689FB001112409
:1011D00040E050E080E0FB01E40FF51FEA56FE4FCF
:1011E000208130E0092E02C0369527950A94E2F757
:1011F00021703327042E01C0220F0A94EAF7822BB4
:101200004F5F5F4F4530510531F70895BF92CF9240
:10121000DF92EF92FF920F931F93CF93DF938C0196
:10122000C090E101D090E201E090E301F090E40190
:101230008091E5019091E601A091E701B091E8016C
:10124000C82AD92AEA2AFB2ACFE1D0E0D701C60171
:101250000C2E04C0B695A795979587950A94D2F75A
:1012600080FD04C0219790F7B12C07C0BC2EB801B7
:101270008C2F0E945A100197A9F38B2DDF91CF91EB
:101280001F910F91FF90EF90DF90CF90BF90089546
:10129000CF93DF93EC010E940609BE010E945A1011
:1012A000DF91CF9108951F93CF93DF93EB0190913E
:1012B0009501992321F0CB010E94480913C088238E
:1012C00049F0CB010E940609182F682FCE010E9419
:1012D000AF0804C0CB010E94DA08182FBE01812F8D
:1012E0000E945A10DF91CF911F9108951F93CF93C1
:1012F000DF93C091E90116E08091EA01C81799F0E7
:10130000D0E01C9FF0011D9FF00D1124E551FE4F10
:101310004081518162817381848195810E948F0710
:101320002196C770E9CFDF91CF911F910895409129
:101330001B0250911C0260911D0270911E0280914F
:101340001F02909120020C948F07EF92FF920F934F
:101350001F93CF93DF938091200282958F7009F0C5
:1013600065C080911D02882309F460C08091E90165
:10137000F090EA0110911B0200911C0260911E0284
:1013800070911F0291E01F3F09F090E0C0910001B1
:10139000D0910101292F96E0E92E8F1509F446C05E
:1013A0006115710521F00F3F21F030E003C031E0FD
:1013B00001C0322F90E030FD36C0E89EF001E99E7A
:1013C000F00D1124DF01A551BE4F11963C911197EC
:1013D000301329C03C91311326C012963C911297CC
:1013E000311121C013964D915C911497461B570BF8
:1013F0004C175D07C0F4809120028F70806180934C
:101400002002E051FE4F80818F70806180838BE1EC
:1014100092E00E940D07DF91CF911F910F91FF90F5
:10142000EF900C94760901968770B7CFDF91CF913A
:101430001F910F91FF90EF9008959F92AF92BF92EE
:10144000CF92DF92EF92FF920F931F93CF93DF9390
:10145000CDB7DEB761970FB6F894DEBF0FBECDBF34
:101460008C0185E0F801DE011D9601900D928A95B0
:10147000E1F7D8011296EC9090911B02E0911C02CA
:1014800020911E0230911F022115310531F0EF3FEE
:1014900031F481E09F3F19F403C081E001C080E096
:1014A000B82FB1709B2E80FD47C1D8014C91119689
:1014B0005C9111971396AD90BC9014978BE1C82E58
:1014C00082E0D82EF0901D02B501621B730B2091B3
:1014D000000130910101FF2009F4D9C08091200260
:1014E0006217730708F095C0282F207F09F052C0BB
:1014F0005E1313C0491311C0FE2CE1100EC08F7093
:101500008061809320020E949709C6010E940D0706
:1015100080912002F80185834DC1AB2831F05F3FF7
:1015200031F481E04F3F19F403C081E001C080E055
:1015300080FD03C081E08E2502C080E090E0F82F9E
:10154000F170FF2E80FF1CC08091E9012091EA011B
:1015500036E0821709F40BC190E0389FF001399F03
:10156000F00D1124E551FE4F6181561306C06081D4
:10157000461303C06281E61203C001968770E9CF6B
:10158000FE2CEE2009F416C1809120028160809328
:10159000200254C05E1306C0491304C0E11002C00B
:1015A000F80199C0C8010E947807882361F1EE20F4
:1015B00051F120912002822F82958F7090E0029746
:1015C00074F080911B0290911C0298878F8319867A
:1015D000BB86AA862C87CE0107960E940D0786E05F
:1015E000F801ABE1B2E001900D928A95E1F70E941B
:1015F000A5090E9497090AC05E1711F1C8010E944F
:10160000780781112CC0C8010E940D07FF24F394B4
:10161000D1C0282F207F81F77A2DB98AA88A6E2D14
:1016200089890E9480078BE192E00E940D0786E085
:10163000D6011D928A95E9F70E949709F12CBAC04C
:101640004913DCCFE110DACFF8018583C8010E948D
:101650000D0786E0D6011D928A95E9F7ABC0EE2012
:1016600091F220912002822F82958F7090E0029754
:101670000CF4B5CF80911B0290911C029A83898350
:101680001B82BD82AC822E83CE010196A6CF62174B
:10169000730708F044C0FE2CEE2009F4B4CF5E13AB
:1016A00030C049132EC02091200220FD21C0822F7E
:1016B00082958F70482F50E041155105C9F0F8010F
:1016C00025834F30510541F08F5F982F9295907F81
:1016D000822F8F70892B8583C8010E940D0786E0B9
:1016E000F801ABE1B2E001900D928A95E1F73CC0C0
:1016F00086E0F801ABE1B2E001900D928A95E1F746
:1017000059C0C8010E947807811169CF80912002D9
:10171000816080932002C8010E940D074BC07A2D82
:10172000B98AA88A6E2D89890E94800786E0D60131
:101730001D928A95E9F718C0EE2009F464CFC8011C
:101740000E947807F82E882309F45DCF86E0F8011F
:10175000ABE1B2E001900D928A95E1F78BE192E066
:101760000E947E030E94A5090E94970923C04D870D
:101770005E878D859E850E944809292F22952F70AE
:10178000223028F49F7039F0811105C00BC024303D
:1017900028F49F7049F4805E883020F0C8010E94D0
:1017A0000D079F2CF92C06C0D80115969C91907FAF
:1017B00091F7F8CF8F2D61960FB6F894DEBF0FBE6C
:1017C000CDBFDF91CF911F910F91FF90EF90DF90F0
:1017D000CF90BF90AF909F9008951F93CF93DF93CA
:1017E000CDB7DEB72C970FB6F894DEBF0FBECDBFD6
:1017F0004F83588769877A878B879C87CE010796A6
:101800000E941D0A8823D1F09F8188852A853B8507
:10181000232B31F08F3F31F481E09F3F19F403C057
:1018200081E001C080E080FD47C04F815885698517
:101830007A858B859C850E948F073EC086E0FE01DD
:101840003796DE01119601900D928A95E1F7FF819E
:10185000E8856A857B856115710531F0EF3F31F4CC
:1018600081E0FF3F19F403C081E001C080E080FD0A
:1018700023C02091EA0130E0C901019687709927C1
:101880004091E90150E084179507F1F1F983EA836B
:101890007D836C8396E0929FD001939FB00D1124BD
:1018A000A551BE4FFE01319601900D929A95E1F738
:1018B0008093EA010E94760916E08091E9019091F7
:1018C000EA01891771F1189FC001112485519E4FBB
:1018D0000E941D0A882329F1E091E9011E9FF00171
:1018E0001124E551FE4F40815181628173818481D1
:1018F00095810E948F078091E90190E001968770A1
:1019000099278093E901D9CF0E9459071092EA01E3
:101910001092E901EBE1F2E086E0DF011D928A9589
:10192000E9F72C960FB6F894DEBF0FBECDBFDF915E
:10193000CF911F9108958091410285958595859558
:1019400008958091410287700895909141029770A7
:1019500081E009F480E008958091640208959091F7
:101960006402892B809364020895809590916402AB
:1019700089238093640208951092640208959091DF
:101980006302892B8093630208958095909163028E
:1019900089238093630208951092630208958091D1
:1019A0004202089508950C94D20C0C94D30C90919B
:1019B000C80292FD08C090914202981721F08093CE
:1019C00042020C94D50C089580914202882329F09C
:1019D0001092420280E00C94D50C0895CF93DF93CF
:1019E000E0910201F0910301809164028083E09113
:1019F0000201F0910301908180916302892B808321
:101A000080914202882381F0E0910201F09103016C
:101A10009081892B808380910201909103010E9423
:101A20001A1881110E94E40CC0910201D0910301A7
:101A300040E250E061E272E0CE010E940221892B77
:101A400069F080E2FE01A1E2B2E001900D928A9578
:101A5000E1F7CE01DF91CF910C94C617DF91CF91C2
:101A600008950C94D20C9091C80292FD10C098E099
:101A7000899F90011124262B209341020E94110876
:101A8000809141028595859585950C94310D0C9436
:101A900011081092410280E00C94310D2091410216
:101AA0008095822380934102982F977099F430E0BB
:101AB000482F082E000C550B2417350759F090912C
:101AC000C80292FD07C08595859585950E943208CC
:101AD0000C94490D08959091C80292FB222720F999
:101AE000281769F080FB92F99093C8028091C70291
:101AF0009091C8020E94B90D82E00C944E0D089599
:101B00008091C80282FB882780F991E089270C9494
:101B10006B0D81E00C946B0D80E00C946B0D6FEFFE
:101B20007FEF80E090E00C943B2180E090E00E9409
:101B3000172121E0893E9E4F09F020E0822F089571
:101B400082E090E00C940F2183E090E00C940F2150
:101B5000CF9384E090E00E940F21C82F82E290E0B2
:101B60000E940F212C2F30E0A901582BCA01CF91E0
:101B70000895CF93C92F682F84E090E00E941D2123
:101B80006C2F82E290E0CF910C941D21AB01BC013F
:101B90008FE090E00C942F21AB01BC0183E190E039
:101BA0000C942F2160E070E0CB010C94CC0D60E030
:101BB00070E0CB010E94C60D0C94D20D69EE7EEF51
:101BC00080E090E00E943B2160E082E090E00E9493
:101BD0001D2160E083E090E00E941D211092E5014C
:101BE0001092E6011092E7011092E80160E084E0B3
:101BF00090E00E941D2160E082E290E00E941D21A1
:101C000060E085E090E00E941D2160E086E090E0C9
:101C10000E941D216FEF87E090E00E941D2140E0AF
:101C200050E0BA0188E090E00E942F2160E08DE052
:101C300090E00E941D2140E050E0BA0188E190E070
:101C40000E942F2160E087E190E00E941D2140E08A
:101C500050E0BA018CE190E00E942F2160E070E03A
:101C600080E290E00E943B2140E050E0BA0188E130
:101C700090E00E942F210C94D70D0C94DE0D682F5C
:101C80008EE090E00C941D210E94801960938102E7
:101C900070938202809383029093840260937D020A
:101CA00070937E0280937F0290938002089585B79F
:101CB000806885BF85B7806885BF089581E00895F5
:101CC0000C945E0E08950C94620E0C94620E0C94AB
:101CD000650E0C94620E0C94690E0C94620E0E94B8
:101CE000570E86E391E10E94B0170E946D0E0C948E
:101CF0006B0E0E94630E0C94620E0E9450110C94A5
:101D000018030E946B190E9435120E947D0EE7ECA9
:101D1000F2E08081806880838091C7029091C80240
:101D20000E94B90D0C94670E5F926F927F928F9212
:101D30009F92AF92BF92CF92DF92EF92FF920F935A
:101D40001F93CF93DF93CDB7DEB72A970FB6F894E2
:101D5000DEBF0FBECDBF0E944A12C82E81110E9465
:101D6000440E35E6832E32E0932E00E010E0502E34
:101D7000802F0E9474115C01F401619071904F01F9
:101D80006826792661147104B1F40F5F1F4F0C307F
:101D9000110569F78FEF89838A831B820E9474196A
:101DA0008160782F9D838C8349815A816B818D81DD
:101DB0000E9434033AC08091850281FD0E947D110A
:101DC000D12CEE24E394F12CC3018E219F21892B89
:101DD00029F10E94600E8823A9F0DE825F82AE2086
:101DE000BF2081E0AB2809F480E088870E94741945
:101DF0008160782F9A8789874E815F8168858A857F
:101E00000E943403000F111FF801EB59FD4F808130
:101E10009181E826F926F182E08207C0D394EE0C86
:101E2000FF1CFAE0DF12D0CFB0CF81E0C11001C0BB
:101E300080E02A960FB6F894DEBF0FBECDBFDF91CB
:101E4000CF911F910F91FF90EF90DF90CF90BF90B7
:101E5000AF909F908F907F906F905F9008950E94B9
:101E6000940E0E9451140C942903CF93DF930E9487
:101E70005F10EC01811521E5920708F045C081153E
:101E800030E5930708F094C0883E910528F5803E20
:101E9000910508F0F8C0883A910570F4853A9105EB
:101EA00008F07CC08130910509F475C008F4E8C0E1
:101EB000049708F0E8C0E4C08F3B910508F0E0C04B
:101EC000C85AD0E0CC0FDD1FC65BDE4F0990D88129
:101ED000C02DCE019464D8C0811540E2940758F417
:101EE000811551E0950708F0CEC08D3E910508F4AC
:101EF000C7C09065C9C0C11580E4D80708F4C0C048
:101F0000DF70CE01906AC0C0811525E59207A8F464
:101F1000811534E5930708F095C0811543E59407D2
:101F200008F07BC0811552E5950708F061C0D82FF5
:101F3000CC27CE01816F906AA7C0C11589E5D8076B
:101F4000A0F4C11528E5D20708F082C0C11536E516
:101F5000D30708F095C08C2F0E94F3108F7190E08A
:101F6000D82FCC27CE0190628FC0C1154AE5D40787
:101F700008F474C0CE0190568115904208F080C0DC
:101F80008D2F8F710E94F310DD27D0628F71AE010B
:101F9000582BCA0179C081E090E076C0C55AD0E0E4
:101FA000C858DE4F8881C82FD0E0CE0190646CC045
:101FB00074E0969587957A95E1F7282F23703C2F4A
:101FC000337081E090E002C0880F991F3A95E2F7E4
:101FD0009C68AC01522B9A019C2F9F709695969508
:101FE00050E2959FE0011124C9018C2B9D2B4CC020
:101FF0008370992721E030E002C0220F331F8A95B9
:10200000E2F79C2F9695969580E2989FE001112427
:10201000C22BD32BCE019C6837C08370992721E057
:1020200030E002C0220F331F8A95E2F79C2F96956D
:10203000969540E2949FE0011124C22BD32BCE0150
:102040009A6822C0D82FCC27CE01846F906A1CC01A
:10205000DC2FCC27CE01806F906A16C08C2F8F703A
:102060000E94F31094E0D695C7959A95E1F7CF704A
:10207000D0E0DC2FCC27D0699E01282BC90104C0F9
:1020800080E090E001C0CE01DF91CF91089528E774
:10209000829FC0011124FC012AE0729FE00DF11D16
:1020A0001124E60FF11DEE0FFF1FE852FF4F85913F
:1020B000949108950E9447100E94350F0895823828
:1020C000910569F1B0F48133910509F46DC048F4CC
:1020D0008932910509F463C08A32910509F469C017
:1020E00008958533910509F455C089339105B9F0F8
:1020F0000895833E910569F138F4803E9105B1F071
:10210000823E910509F10895863E9105A9F1873E29
:102110009105B9F1843E910509F064C023C0209176
:10212000C70220FD4FC021FD4DC008958091C70218
:1021300080FD44C08091C80280FF44C08091C702E6
:1021400084FD42C083EE4DC08091C70282FF38C03B
:10215000F5CF8091C70282FD33C08091C80280FD17
:1021600031C0ECCF8091C80281FF32C08091C7029C
:1021700084FD2AC087EE35C08091C70283FF26C048
:10218000F5CF8091C70283FD21C08091C80281FDF7
:102190001FC0ECCF8091C70285FD1CC01DC080917F
:1021A000C70285FD19C016C08091C70286FD16C002
:1021B00017C08091C70286FD13C010C089E311C00B
:1021C00082EE0FC080EE0DC080E00BC086EE09C02D
:1021D00084EE07C089E205C085E303C08AE201C03E
:1021E00081E390E008959091C70292FF0DC0282FDF
:1021F0002871283019F4877F846006C0282F247145
:10220000243011F48B7F886093FF0DC0282F287134
:10221000283119F4877E846106C0282F2471243167
:1022200011F48B7E88612091C80220FF0DC0382FE9
:102230003871383019F4877F816006C0382F3171CA
:10224000313011F48E7F886021FF0DC0282F287156
:10225000283119F4877E816106C0282F2171213130
:1022600011F48E7E886194FD877E089580E0089544
:102270000C948F0D0E944A128FE39CE90197F1F7AD
:1022800000C000000E944A1280E00E94741180FF8A
:1022900004C00E9438110C94C11908950C943A118D
:1022A0000E94950D811102C00E943D0E0E94A00D5A
:1022B000809385020E94A80D9093C8028093C70264
:1022C0000E944E110E94A40D682F70E080E090E003
:1022D0000E94B1076091E1017091E2018091E301F8
:1022E0009091E4010C94E907E82FF0E0EE0FFF1F56
:1022F000EF51FD4F808191810895089580EA8A957C
:10230000F1F7089500C008950C947E1108950C947F
:1023100086110C9487110C9486110C948B11F894EF
:10232000E82FE295EF70F0E031A1282F2F7081E0C7
:1023300090E001C0880F2A95EAF7982F9095932393
:1023400091A392A1892B82A3789408950F931F9350
:10235000CF93DF93C5E8D1E089918F3F11F00E94C0
:102360008F1181E0C139D807B9F7CBE7D1E005E893
:1023700011E089918F3F11F00E948F110C171D07FA
:10238000C1F7DF91CF911F910F910895BF92CF9226
:10239000DF92EF92FF920F931F93CF93DF938C0105
:1023A000C62FD0E0CE018B579E4F6C01FC0190816F
:1023B0009F3F09F450C0B62EF894E92FE295EF70D4
:1023C000F0E081A19F7021E030E001C0220F9A95DA
:1023D000EAF7822B81A382A12095282322A3789457
:1023E0000E948211EBE7F1E045E851E021E030E0A6
:1023F000E12CF12C61916F3F89F0A62FA295AF706F
:10240000B0E090968C9190E06F7002C095958795A2
:102410006A95E2F780FD02C0C90102C080E090E049
:10242000E82AF92A220F331F4E175F0719F7F60122
:1024300080818F3F11F00E948F1161E0E114F1045F
:1024400009F460E08B2D0E948411CC0FDD1FC00FBA
:10245000D11FF982E882DF91CF911F910F91FF90F8
:10246000EF90DF90CF90BF9008950E94A61188E171
:10247000E1EEF2E0DF01982F1D929A95E9F7E9EC81
:10248000F2E0DF011D928A95E9F78CE00E94951237
:102490000C94A402FF920F931F93CF93DF93CDB7B9
:1024A000DEB768970FB6F894DEBF0FBECDBF8E01C2
:1024B0000F5F1F4F88E1F80111928A95E9F7F12C1F
:1024C0006F2DC8010E94C611F394FCE0FF12F8CFF3
:1024D00048E150E0B80189EC92E00E940221FF241B
:1024E000F394009709F4F12C892B41F088E1F8016D
:1024F000A9ECB2E001900D928A95E1F72F2D4CE006
:1025000061EE72E089EC92E00E9496120E94A602AF
:102510008F2D68960FB6F894DEBF0FBECDBFDF914A
:10252000CF911F910F91FF9008950895FF920F93FF
:102530001F93CF93DF93F82E092F162FD72FC42F79
:10254000222349F081E0809388020E9474199093BD
:10255000870280938602809188028823D9F0809137
:102560008602909187020E948C19059798F0EF2DB2
:10257000F02FA12FBD2F80E090E04C2F50E084176A
:10258000950734F4219131912D933D930196F7CF26
:1025900010928802DF91CF911F910F91FF900895C3
:1025A0000E949A1B0E94810E0C94A61B0E94AA1BDB
:1025B0000E942F0F0C94C41B0E9412190E94811BB1
:1025C0000E946F0E0E94D0120E94D6120E94790EB5
:1025D000FBCF80918F0280FF06C06091090170E0FF
:1025E000660F771F26C081FF04C06091090184E057
:1025F00005C082FF07C06091090188E0689FB001B3
:10260000112417C090918E029923D1F06091080196
:10261000961788F72091090188E0289F90011124DE
:10262000929FA001939F500D112470E0CA010E9457
:10263000D4206038710540F46115710519F406C0A5
:1026400068E070E0862F08958FE7089581E008958F
:1026500080918F0280FF08C06091050170E0759540
:1026600067957595679521C081FF06C0609105014A
:1026700070E07595679519C082FF04C060910501EF
:1026800070E010C090918D02992399F0609104013F
:102690009617A0F780910501899FC001112470E071
:1026A0000E94D4206038710540F46115710519F459
:1026B00006C061E070E0862F08958FE7089581E0FD
:1026C00008958D3E21F40E94E912819504C08E3E4A
:1026D00029F40E94E9128093930208958F3E21F419
:1026E0000E94E912819504C0803F29F40E94E912FA
:1026F000809392020895893F19F40E94281305C01F
:102700008A3F31F40E9428138195809394020895A2
:102710008B3F21F40E942813819504C08C3F29F43B
:102720000E9428138093950208959FE0980F983097
:1027300078F421E030E0A90102C0440F551F9A95BA
:10274000E2F7CA0190919102892B8093910208953A
:102750008D3F21F480918F0281600BC08E3F21F468
:1027600080918F02826005C08F3F29F480918F0293
:10277000846080938F0208958D3E39F49091930286
:1027800097FF35C01092930259C08E3E29F4909164
:1027900093021916BCF32BC0909192028F3E29F43C
:1027A00097FF25C01092920249C0803F19F4191674
:1027B000CCF31DC090919402893F29F41916BCF402
:1027C000109294023BC08A3F19F497FF10C0F8CFD3
:1027D0008B3F39F49091950297FF09C010929502B2
:1027E0002DC08C3F21F4909195021916BCF39FE007
:1027F000980F983080F421E030E0A90102C0440F26
:10280000551F9A95E2F7CA0180959091910289230C
:102810008093910213C08D3F21F480918F028E7FAF
:102820000BC08E3F21F480918F028D7F05C08F3FBA
:1028300029F480918F028B7F80938F028091920286
:10284000811106C080919302811102C010928E0204
:1028500080919402811106C080919502811102C07D
:1028600010928D0208950E947419209192022111F4
:1028700004C020919302222321F090938C02809334
:102880008B0220919402211104C0209195022223F1
:1028900021F090938A028093890280E992E00C945F
:1028A000E017EF92FF920F931F93CF93DF9300D027
:1028B00000D000D0CDB7DEB786E0E0E9F2E0DE017F
:1028C000119601900D928A95E1F7E0909202F090B6
:1028D000930200919402109195021092920210922C
:1028E00093021092940210929502E11003C0FF200F
:1028F00009F45DC080918B0290918C020E948C192A
:10290000AC0190918E02992339F020910A0130E0B8
:102910002417350758F04BC020910B018AE0289FFF
:10292000900111242417350718F041C09F3F19F07A
:102930009F5F90938E02EE2061F00E94E9121E14B8
:1029400014F09FEF01C091E0989F902D1124909377
:102950009202FF2061F00E94E9121F1414F09FEF11
:1029600001C091E0989F902D112490939302309193
:1029700092023323E1F0209193022223C1F045EB30
:102980003403C0011124992319F09093920203C0DB
:1029900081E08093920235EB2303C0011124992337
:1029A00019F09093930203C081E080939302011188
:1029B00003C0112309F45DC08091890290918A02BD
:1029C0000E948C19AC0190918D02992339F02091CD
:1029D000060130E02417350758F04BC0209107015D
:1029E0008AE0289F900111242417350718F041C070
:1029F0009F3F19F09F5F90938D02002361F00E942A
:102A00002813101614F09FEF01C091E0989F902DAD
:102A1000112490939402112361F00E94281311163F
:102A200014F09FEF01C091E0989F902D1124909396
:102A30009502309194023323E1F0209195022223F4
:102A4000C1F045EB3403C0011124992319F0909390
:102A5000940203C081E08093940235EB2303C0010C
:102A60001124992319F09093950203C081E080937B
:102A700095028091920281110BC080919302811185
:102A800007C080919402811103C080919502811149
:102A90000E943314EB82FC820D831E8386E0FE01CC
:102AA0003196A0E9B2E001900D928A95E1F7269661
:102AB0000FB6F894DEBF0FBECDBFDF91CF911F914F
:102AC0000F91FF90EF900895E0E9F2E086E0DF01DA
:102AD0001D928A95E9F710928E0210928D02109243
:102AE0008F020895CF93DF93EC01FB01828188234D
:102AF00009F43CC1C430FDE5DF0760F4CB3F9CE541
:102B0000D90788F49E0122503C452431310508F054
:102B10002EC109C0C236EDE5DE0729F0C63AFDE553
:102B2000DF0709F024C10E94A80D9093C80280938A
:102B3000C702C1318CE5D80709F4C6C008F042C00D
:102B4000C930ECE5DE0709F49BC000F5C5308CE523
:102B5000D80709F485C078F4C330ECE5DE0709F442
:102B600078C008F07AC0C230DC4509F0F5C0809129
:102B7000C7028160EFC0C7309CE5D90709F478C06F
:102B800008F07AC08091C7028061E4C0CD30FCE5D6
:102B9000DF0709F487C058F4CB309CE5D90709F466
:102BA00079C008F07BC08091C70288606FC0CF30C9
:102BB000FCE5DF0709F480C008F082C08091C702FD
:102BC000877FC8C0CE3F9CE5D90709F471C000F5E6
:102BD000C531FCE5DF0709F485C068F4C3319CE525
:102BE000D90709F475C008F095C00E945907809173
:102BF000C7028F77AFC0CC3FFCE5DF07A9F108F033
:102C000054C0CB3FDC4509F0A7C08091C80240C04A
:102C1000C230EDE5DE0709F489C058F4C1158DE531
:102C2000D80709F45AC008F069C08091C8028260D0
:102C30002FC0C236EDE5DE0709F47CC0C63AFDE5DB
:102C4000DF0709F481C0C330DD4509F085C080E0AD
:102C50006EC08091C70282607DC08091C70216C09D
:102C60008091C702886076C08091C80282604FC0A0
:102C70008091C70280626EC08091C70280646AC082
:102C80000E9459078091C702806864C0846062C056
:102C900081603DC08091C7028E7F5CC08091C70279
:102CA0008D7F58C08091C70216C08091C80218C09D
:102CB0008091C8028D7F2BC08091C7028F7E4AC051
:102CC0008091C7028F7D46C08091C7028F7B42C032
:102CD0008091C702877F8B7F3DC08091C8028D7F26
:102CE0008E7F15C08091C70282FB222720F991E0D8
:102CF000922790FB82F990FB83F92CC08091C80247
:102D0000982F909591708E7F892B90FB81F98093FD
:102D1000C80222C00E9459078091C70287FB222760
:102D200020F991E0922790FB87F914C081E00E947E
:102D30003F0E12C08091C70284FB222720F991E048
:102D4000922790FB84F906C08091C702982F909536
:102D500090FB80F98093C7028091C7029091C802CE
:102D60000E94B90D0E94590780E001C081E0DF9107
:102D7000CF910895CF93DF9386319C4541F5EB01C8
:102D80000E94AC0C982F8A8120910201309103019E
:102D9000882379F09A7A81E009F480E080939602A2
:102DA000911102C069E201C065E3C9010E94B01837
:102DB0000AC080919602811102C069E201C065E3F8
:102DC000C9010E94BB180E94EE0C80E001C081E0A6
:102DD000DF91CF9108950F931F93CF93DF93C42F6B
:102DE000D22FFC0182818823C9F0409399020E946E
:102DF0007419909398028093970280E28C0F883028
:102E000008F057C0C77081E001C0880FCA95EAF783
:102E1000DF91CF911F910F910C94B604809199028C
:102E2000481330C080919702909198020E948C19AB
:102E3000883C910538F510E21D0FCD17B9F080E2FE
:102E40008C0F883040F4C77081E001C0880FCA95AC
:102E5000EAF70E94BD04183028F581E09D2F977095
:102E600001C0880F9A95EAF70E94B604802F0E944D
:102E7000AD041830F0F4D77081E001C0880FDA9506
:102E8000EAF70AC080E28C0F883098F4C77081E0BE
:102E900001C0880FCA95EAF7DF91CF911F910F917A
:102EA0000C94BD04802FDF91CF911F910F910C9452
:102EB000AD04DF91CF911F910F9108950F939C0165
:102EC000CB01243F4CE5340731F188F4293DFCE582
:102ED0003F07D9F02A3D4CE5340779F1283D3C45C0
:102EE000A9F506E221EE41EE68ED7CE52BC0263F18
:102EF000FCE53F07E1F0A8F0273F3C4539F507E244
:102F000025EE46EE67EF7CE51DC007E225EE45EEB7
:102F100069ED7CE517C006E221EE40EE64EF7CE54A
:102F200011C007E225EE44EE65EF7CE50BC006E23A
:102F300021EE42EE66EF7CE505C008E221E045EEB9
:102F40006AED7CE50E94EB1680E008C0FC018281FE
:102F5000882319F01092990201C081E00F91089521
:102F60009093930180939201089590939F02809390
:102F70009E020895E0919E02F0919F02309721F009
:102F80000190F081E02D099480E00895E0919E0287
:102F9000F0919F02309799F020911801222359F067
:102FA0002091C70227FF07C0DC012C9111962C93BA
:102FB000119726E02C930280F381E02D0994089567
:102FC000E0919E02F0919F02309739F022E0DC01FF
:102FD0002C930480F581E02D0994089520919C02A2
:102FE00030919D022817390771F090939D028093CC
:102FF0009C02E0919E02F0919F02309721F00680A2
:10300000F781E02D0994089520919A0230919B0256
:103010002817390771F090939B0280939A02E091F0
:103020009E02F0919F02309721F00084F185E02DFF
:1030300009940895FC01329680911801882331F09B
:103040008091C70287FF02C09EE101C096E080E048
:10305000915028F021912223D9F38F5FF9CF089561
:10306000662351F1209118012223E9F02091C70233
:1030700027FF19C0462F4695469546954E31E0F4F8
:10308000677021E030E002C0220F331F6A95E2F73B
:10309000FC01E40FF11D828190E02823392381E0B7
:1030A000232B69F409C0FC0132960896219162171E
:1030B00029F0E817F907D1F780E0089581E0089535
:1030C0009C01FC0132969FEF80E04191461789F008
:1030D0009F3F19F4411101C0982F8F5F8630A9F7E7
:1030E0009F3F39F0F901E90FF11D97FDFA956283D1
:1030F000089508959C012A5F3F4FFC0142814613C9
:1031000001C01282019682179307B9F70895262FFE
:103110002695269526952E3168F4FC01E20FF11DC7
:10312000677021E030E001C0220F6A95EAF78281E2
:10313000282B22830895262F2695269526952E3115
:1031400070F4FC01E20FF11D677021E030E001C076
:10315000220F6A95EAF72095828128232283089519
:1031600020911801222329F02091C70227FD0C94F9
:1031700087180C94601820911801222329F02091BF
:10318000C70227FD0C949B180C947A182091180103
:10319000FC013296222331F08091C70287FF02C0E2
:1031A0008EE101C086E0DF011D928A95E9F708955E
:1031B00008950C94D81883E08093A0020C94D91839
:1031C000811102C081E001C082E08093A0020C94D2
:1031D000D9180C94E01881E08093A0020C94D918BF
:1031E0000C94EB1808950C94F2180C94F3180C94AA
:1031F000F2180C94F2180C94F218CF930E94F9185C
:103200000E944A120E94F718C0E08C2F0E9474118D
:10321000892B29F4CF5FCC30C1F780E001C081E079
:10322000CF91089508951F920F920FB60F92112417
:103230008F939F93AF93BF938091A102811113C08D
:103240008091F9029091FA02A091FB02B091FC02E8
:103250004196A11DB11D8093F9029093FA02A093AB
:10326000FB02B093FC02BF91AF919F918F910F90A1
:103270000FBE0F901F90189580910103843031F19B
:103280000E940A031092A10220E488E190E00FB6A8
:10329000F894A895809360000FBE2093600083B7D8
:1032A000817F846083BF83B7816083BF7894889572
:1032B00083B78E7F83BF0FB6F894A8958091600086
:1032C000886180936000109260000FBE08950E9494
:1032D00059070C940E0382E084BD93E095BD9AEFEC
:1032E00097BD80936E0008952FB7F8948091F902EE
:1032F0009091FA02A091FB02B091FC022FBF0895B9
:103300002FB7F8946091F9027091FA028091FB0254
:103310009091FC022FBF08959C014FB7F8948091C3
:10332000F9029091FA02A091FB02B091FC024FBF0A
:10333000821B930B089578941F920F920FB60F92F1
:1033400011248F939F93AF93BF938091F902909133
:10335000FA02A091FB02B091FC020196A11DB11DE1
:103360008093F9029093FA02A093FB02B093FC02BF
:10337000BF91AF919F918F910F900FBE0F901F90B3
:103380001895F89481E08093E00080E28093D80063
:10339000E9ECF0E010828FE19EE40197F1F700C0C4
:1033A00000001DBA109268001CBC10BE1FBA10921B
:1033B0007A0010926E0010926F00109271001092BD
:1033C00072001082ECEBF0E0108214B817B81AB853
:1033D0001DB810BA108215B818B81BB81EB811BAAB
:1033E0000C94003F08958091C5020895089522E04D
:1033F0002093E9002FEF3091E800215035FD06C001
:1034000035ED3A95F1F700002111F5CF2091E80054
:1034100025FF0BC040E050E066E070E00E94361CE3
:103420008091E8008E778093E8000895CF93DF9332
:1034300020911801222339F02091C70227FF03C0F1
:1034400060E222E002C068E021E02093E9002FEF73
:103450003091E800215035FD06C035ED3A95F1F781
:1034600000002111F5CF2091E80025FF1DC0EC01DF
:1034700080911801811105C040E050E068E070E0E3
:1034800003C070E040E050E0CE010E94361C809105
:10349000E8008E778093E80080E2FE01A5EAB2E0C2
:1034A00001900D928A95E1F7DF91CF910895809375
:1034B000A2027093A4026093A3028091010384305E
:1034C00001F582E08093E9008FEF9091E800815050
:1034D00095FD06C095ED9A95F1F700008111F5CFA5
:1034E0008091E80085FF0DC040E050E063E070E0AF
:1034F00082EA92E00E94361C8091E8008E778093E9
:10350000E8000895BC0184E00C94571ABC0183E0E4
:103510000C94571A80910003811109C00E94C71DA5
:103520000E94241E8091E20084608093E20008954E
:103530001092000308950C94F0186091FD0281E050
:10354000611101C080E00C94DB189091010381E0CF
:10355000943009F080E06091FD020C94E01842E0A4
:1035600061EC81E00E94401D42E261EC82E00E9439
:10357000401D9091010381E0943009F080E060915A
:10358000FD020C94E91880910303833009F461C0B3
:1035900030F4813071F0823009F49AC008958A3095
:1035A00009F486C08B3009F46CC0893009F0A8C0DA
:1035B00020C080910203813A09F0A2C08091E80006
:1035C000877F8093E8008091060390910703892B01
:1035D00021F460E285EA92E003C060E080E090E0E0
:1035E00070E00E94811C8091E8008B778093E80056
:1035F000089580910203813209F082C08091060310
:1036000090910703029708F07BC08091E800877FC4
:103610008093E8008091E80082FD05C0809101035D
:103620008111F8CF6DC02091F3008091F20090E0FD
:10363000922B029731F48091F100813011F08630A5
:1036400021F48091F1008093C5028091E8008B778E
:1036500053C080910203813A09F052C08091060361
:1036600090910703892B09F04BC08091E800877F78
:103670008093E8008091E80080FFFCCF80911801E2
:1036800036C0809102038132D9F580910603909172
:103690000703892BA9F58091E800877F8093E800D4
:1036A0000E94751D80910403809318010C945907A2
:1036B00080910203813221F58091E800877F809319
:1036C000E8000E94751D809105038093C60208954D
:1036D00080910203813AA1F48091E800877F809372
:1036E000E8008091E80080FFFCCF8091C6028093C3
:1036F000F1008091E8008E778093E8000C94751DAE
:10370000089584B7877F84BF0FB6F894A8958091F9
:103710006000886180936000109260000FBE90E0AE
:1037200080E80FB6F89480936100909361000FBE1B
:103730000C94EB180E94C71D0E94241EE2EEF0E0DC
:1037400080818460808378940C94B9208CE091E02F
:103750000C94B517809101038530A9F48091010381
:10376000853079F40E943C198091FF028823B1F3DF
:103770000E94FD18882391F30E94201C0E94590783
:10378000EDCF0C946719089508950C94C71B292F49
:10379000332723303105C9F060F42130310581F041
:1037A0002230310509F044C08BE390E02CEF32E089
:1037B00043C021323105E1F02232310549F138C0F0
:1037C00082E190E027E333E037C09927813091050B
:1037D00049F028F0029761F5E8EBF2E005C0E8EF68
:1037E000F2E002C0E4EDF2E0849190E09F0124C099
:1037F0006115710541F061307105D1F489E090E007
:1038000027E233E019C089E090E02EE033E014C0F5
:103810006115710541F06130710551F486EB90E05E
:1038200029E433E009C080E490E02FEF33E004C0E6
:1038300080E090E020E030E0FA01318320830895B9
:1038400080E189BD82E189BD09B400FEFDCF809190
:10385000D8008F7D8093D8008091E00082608093B3
:10386000E0008091E00081FDFCCF0895CF92DF92CF
:10387000EF92FF920F931F93CF93DF93EC018B0195
:103880007A010E94941D811133C0E114F10439F0D2
:10389000F70180819181081B190BC80FD91FC12C1A
:1038A000D12C0115110519F18091E80085FD16C094
:1038B0008091E8008E778093E800E114F10449F0EC
:1038C000F70180819181C80ED91ED182C08285E026
:1038D0000FC00E94941D882321F30AC08991809310
:1038E000F10001501109FFEFCF1ADF0ADACF80E0B3
:1038F000DF91CF911F910F91FF90EF90DF90CF90CC
:10390000089520910803309109032617370748F0DE
:103910006115710539F42091E8002E772093E800B5
:1039200001C0B901FC0120E06115710579F18091B8
:1039300001038823F1F18530F1F18091E80083FDE6
:103940003CC08091E80082FD2EC08091E80080FF9D
:10395000EBCF2091F3008091F20090E0922B611563
:10396000710551F08830910538F421912093F100D0
:10397000615071090196F3CF21E0089709F020E02A
:103980008091E8008E778093E800CECF2111CFCFD1
:103990000AC080910103882361F0853061F0809135
:1039A000E80083FD0AC08091E80082FFF2CF80E04A
:1039B000089582E0089583E0089581E008952091BC
:1039C0000803309109032617370748F06115710580
:1039D00039F42091E8002E772093E80001C0B90166
:1039E000FC0120E06115710591F1809101038823AC
:1039F00009F440C0853009F43FC08091E80083FDA0
:103A00003DC08091E80082FD2FC08091E80080FFDA
:103A1000E9CF2091F3008091F20090E0922B6115A4
:103A2000710559F08830910540F424912093F100FC
:103A30003196615071090196F2CF21E0089709F0A3
:103A400020E08091E8008E778093E800CBCF2111B1
:103A5000CCCF0AC080910103882361F0853061F0EA
:103A60008091E80083FD0AC08091E80082FFF2CFD8
:103A700080E0089582E0089583E0089581E008954C
:103A8000982F973068F59093E900981739F0709166
:103A9000EC002091ED005091F00003C0242F762F10
:103AA00050E021FD02C09F5FECCF3091EB003E7FE4
:103AB0003093EB003091ED003D7F3093ED0030917D
:103AC000EB0031603093EB007093EC002093ED003D
:103AD0005093F0002091EE0027FDE5CF80E008959F
:103AE0008F708093E90081E008958091020387FF41
:103AF00011C08091E80082FD05C080910103811111
:103B0000F8CF11C08091E8008B770BC08091010342
:103B1000882349F08091E80080FFF8CF8091E80089
:103B20008E778093E80008952091E4003091E500BD
:103B300095E64091EC00842F817040FF23C0809176
:103B4000E80080FD1DC080910103882399F0853035
:103B500099F08091EB0085FD11C04091E4005091F7
:103B6000E5002417350729F3915011F09A01E1CFB0
:103B700084E0089582E0089583E0089581E0089547
:103B800080E008954091E80042FFDDCF08950E9453
:103B9000351E0E943D1EE0EEF0E080818160808352
:103BA000E8EDF0E080818F77808319BCA7EDB0E06D
:103BB0008C918E7F8C9380818F7E80831092000306
:103BC00008950F931F93CF93DF930E94351E0E9499
:103BD0003D1EC8EDD0E088818F778883888180681A
:103BE000888388818F7D888319BC1092010310928D
:103BF000FD021092FF021092FE0200EE10E0F801AA
:103C000080818B7F808388818160888342E060E04F
:103C100080E00E94401DE1EEF0E080818E7F808395
:103C2000E2EEF0E080818160808380818860808323
:103C3000F80180818E7F8083888180618883DF9115
:103C4000CF911F910F910895E8EDF0E080818F7E74
:103C50008083E7EDF0E080818160808384E082BF33
:103C600081E0809300030C94E11DE8EDF0E0808199
:103C70008E7F80831092E20008951092DA001092F5
:103C8000E10008951F920F920FB60F9211242F9307
:103C90003F934F935F936F937F938F939F93AF93D4
:103CA000BF93EF93FF938091E10082FF0BC080915F
:103CB000E20082FF07C08091E1008B7F8093E100EA
:103CC0000E94B8208091DA0080FF1FC08091D80048
:103CD00080FF1BC08091DA008E7F8093DA00809194
:103CE000D90080FF0DC080E189BD82E189BD09B4A2
:103CF00000FEFDCF81E0809301030E948A1A05C077
:103D000019BC109201030E94981A8091E10080FF73
:103D100019C08091E20080FF15C08091E2008E7F83
:103D20008093E2008091E20080618093E2008091C4
:103D3000D80080628093D80019BC85E0809301038D
:103D40000E949D1A8091E10084FF30C08091E200C2
:103D500084FF2CC080E189BD82E189BD09B400FEE9
:103D6000FDCF8091D8008F7D8093D8008091E100B5
:103D70008F7E8093E1008091E2008F7E8093E2004D
:103D80008091E20081608093E2008091FD028823AF
:103D900011F084E007C08091E30087FD02C081E05C
:103DA00001C083E0809301030E94A51A8091E10085
:103DB00083FF29C08091E20083FF25C08091E1004C
:103DC000877F8093E10082E0809301031092FD02DF
:103DD0008091E1008E7F8093E1008091E2008E7FF0
:103DE0008093E2008091E20080618093E20042E0F3
:103DF00060E080E00E94401D8091F0008860809328
:103E0000F0000E949B1AFF91EF91BF91AF919F919B
:103E10008F917F916F915F914F913F912F910F9073
:103E20000FBE0F901F9018951F920F920FB60F9212
:103E300011242F933F934F935F936F937F938F93AF
:103E40009F93AF93BF93CF93DF93EF93FF93C09173
:103E5000E900CF708091EC00D82FD17080FDD0E8C0
:103E60001092E9008091F000877F8093F0007894B1
:103E70000E94581F1092E9008091F00088608093A2
:103E8000F000CD2BCF70C093E900FF91EF91DF914F
:103E9000CF91BF91AF919F918F917F916F915F91E2
:103EA0004F913F912F910F900FBE0F901F9018953B
:103EB0001F93CF93DF93CDB7DEB7AA970FB6F894D1
:103EC000DEBF0FBECDBFE2E0F3E08091F100819351
:103ED00023E0EA30F207C9F70E94C31A8091E80094
:103EE00083FF2EC18091020390910303492F50E07C
:103EF0004A30510508F024C1FA01EE59FF4F0C94E5
:103F0000E820803821F0823809F01AC108C0809179
:103F1000FE029091FF02992389F082600FC0809188
:103F200006038F70873008F00BC18093E900809101
:103F3000EB0085FB882780F91092E9009091E8005A
:103F4000977F9093E8008093F1001092F100D1C028
:103F5000282F2D7F09F0F4C0882319F0823061F0FA
:103F6000EFC080910403813009F0EAC0933009F07A
:103F700080E08093FF022EC08091040381112AC04B
:103F8000809106038F702FEF280F263008F0D8C0DD
:103F90008093E9002091EB0020FF1CC0933021F4B6
:103FA0008091EB00806214C09091EB00906190933F
:103FB000EB0021E030E0A90102C0440F551F8A95B3
:103FC000E2F74093EA001092EA008091EB008860EB
:103FD0008093EB001092E9008091E800877F809346
:103FE000E8000E94751DACC08111AAC010910403A5
:103FF0001F778091E3008078812B8093E30080918C
:10400000E800877F8093E8000E94751D8091E8009A
:1040100080FFFCCF8091E30080688093E300111162
:1040200002C082E001C083E08093010389C0805810
:10403000823008F085C080910403909105038C3D87
:1040400053E0950779F583E08A838AE289834FB745
:10405000F894DE01139620E03EE051E2E32FF0E019
:1040600050935700E49120FF03C0E295EF703F5F4B
:10407000EF708E2F90E0EA3010F0C79601C0C09626
:104080008D939D932F5F243149F74FBF8091E800B6
:10409000877F8093E8006AE270E0CE0101960E947B
:1040A000811C16C06091060370910703AE014F5F3B
:1040B0005F4F0E94C51BBC01892B09F441C0909140
:1040C000E800977F9093E80089819A810E94DF1C25
:1040D0008091E8008B778093E80032C0803881F5CA
:1040E0008091E800877F8093E8008091FD028093B3
:1040F000F1008091E8008E7772CF811121C080910C
:1041000004039091050399270297D4F48091E80065
:10411000877F8093E800809104038093FD020E94D2
:10412000751D8091FD02811106C08091E30087FD1D
:1041300002C081E001C084E0809301030E94AF1AB5
:104140008091E80083FF0AC08091E800877F809318
:10415000E8008091EB0080628093EB00AA960FB696
:10416000F894DEBF0FBECDBFDF91CF911F910895B0
:104170000895CF93809101038823A1F0C091E900B5
:10418000CF709091EC00892F817090FD80E8C82B52
:104190001092E9008091E80083FD0E94581FCF70C3
:1041A000C093E900CF91089597FB072E16F4009471
:1041B00007D077FD09D00E94EE2007FC05D03EF421
:1041C000909581959F4F0895709561957F4F0895C3
:1041D000EE0FFF1F0590F491E02D0994AA1BBB1B65
:1041E00051E107C0AA1FBB1FA617B70710F0A61BF7
:1041F000B70B881F991F5A95A9F780959095BC0118
:10420000CD010895FB01DC0104C08D91019080195E
:1042100021F441505040C8F7881B990B0895F99933
:10422000FECF92BD81BDF89A992780B50895A8E187
:10423000B0E042E050E00C944321262FF999FECFE4
:1042400092BD81BDF89A019700B4021639F01FBAE9
:1042500020BD0FB6F894FA9AF99A0FBE0895039606
:10426000272F0E941E210E941D21252F0E941E2102
:10427000242F0C941E210196272F0E941E210C949E
:104280001D21DC01CB01FC01F999FECF06C0F2BD76
:10429000E1BDF89A319600B40D9241505040B8F704
:0642A0000895F894FFCF21
:1042A600C8004302280850011E0A1401F319161A01
:1042B600F719861A821AF61901E200E900EA00B532
:1042C60000B600B700CD008301CC008A01920194AC
:1042D600012102230224022502260227022A02B312
:1042E60000B4006F007000818283E200E900EA00FA
:1042F600B500B600B700CD008301CC008A0192015B
:1043060094012102230224022502260227022A0200
:10431600B300B4006F00700081828391903733320E
:104326003130C69293F0F1F494F6F5F73635956789
:0243360066001F
:00000001FF
